:020000040800F2
:1000000000000320755000082D0C00082F0C00087C
:10001000310C0008330C0008350C0008000000000B
:10002000000000000000000000000000370C000885
:10003000390C0008000000003B0C00083D0C0008D3
:10004000C5500008C5500008C5500008C55000083C
:10005000C5500008C5500008450C0008C5500008F0
:10006000C5500008810C0008C5500008C5500008A4
:10007000C5500008C5500008C5500008C55000080C
:10008000C5500008C5500008C5500008C5500008FC
:10009000C5500008C5500008C5500008C5500008EC
:1000A000C5500008C5500008C5500008C5500008DC
:1000B000C5500008C5500008C5500008C5500008CC
:1000C000C5500008C5500008C5500008C5500008BC
:1000D000C5500008C5500008C5500008C5500008AC
:1000E000C5500008C5500008C5500008C55000089C
:1000F000C5500008C5500008C5500008C55000088C
:10010000C5500008C5500008C5500008C55000087B
:10011000C5500008C5500008C5500008C55000086B
:10012000990C0008C5500008C5500008C5500008CB
:10013000C5500008C5500008C5500008C55000084B
:10014000C5500008C5500008C5500008A90C00089B
:10015000C5500008C5500008C5500008C55000082B
:10016000C5500008C5500008C5500008C55000081B
:10017000C5500008C5500008C55000080000000028
:10018000C5500008C5500008C5500008C5500008FB
:10019000C5500008C5500008C5500008C5500008EB
:0C01A000C5500008C5500008C5500008FC
:1001B0000348044B834202D0034B03B118477047F6
:1001C0001C0100201C010020000000000548064B17
:1001D0001B1AD90F01EBA301491002D0034B03B145
:1001E000184770471C0100201C010020000000007F
:1001F00010B5064C237843B9FFF7DAFF044B13B16F
:100200000448AFF300800123237010BD1C010020BF
:1002100000000000C850000808B5044B1BB1044999
:100220000448AFF30080BDE80840CFE700000000BD
:1002300020010020C850000870B50F4B0F4DAB4295
:10024000A3EB050607D0B610002455F8043B013493
:100250009847A642F9D804F037FF094D094B5E1BB9
:10026000AB424FEAA60606D0002455F8043B013401
:100270009847A642F9D870BD485100084851000877
:10028000485100084C510008830730B547D0541E30
:10029000002A3ED0CAB2034601E0013C39D303F83C
:1002A000012B9D07F9D1032C2CD9CDB205EB0525E7
:1002B0000F2C05EB054535D9A4F1100222F00F0CE7
:1002C00003F1100EE6444FEA121C1A46C2E900552B
:1002D000C2E9025510327245F8D10CF1010214F056
:1002E0000C0F03EB021204F00F0C13D0ACF104035B
:1002F00023F003030433134442F8045B9342FBD11D
:100300000CF003042CB1C9B21C4403F8011BA34236
:10031000FBD130BD64461346002CF4D1F9E7034607
:100320001446C0E71A46A446E0E700BF7BB972B99D
:100330000029BEBF00204FF0004106E008BF0028A2
:100340001CBF6FF000414FF0FF3000F0B5B9ADF1C8
:10035000080C6DE904CE002909DB002B1ADB00F044
:100360004DF8DDF804E0DDE9022304B070474042B7
:1003700061EB4101002B1BDB00F040F8DDF804E0ED
:10038000DDE9022304B0404261EB4101524263EBDC
:1003900043037047524263EB430300F02FF8DDF84C
:1003A00004E0DDE9022304B0404261EB4101704703
:1003B000524263EB430300F021F8DDF804E0DDE98D
:1003C000022304B0524263EB4303704753B94AB966
:1003D000002908BF00281CBF4FF0FF314FF0FF304D
:1003E00000F06AB9ADF1080C6DE904CE00F006F832
:1003F000DDF804E0DDE9022304B070472DE9F047A1
:10040000089D0E4604460F46002B4AD194468C4563
:10041000B2FA82F260D942B1C2F12003974020FAC9
:1004200003F30CFA02FC1F4394404FEA1C4E1FFAE0
:100430008CF6B7FBFEF1230C0EFB117743EA074362
:1004400001FB06F098420AD91CEB030301F1FF37C8
:1004500080F01581984240F21281023963441B1AE0
:10046000A4B2B3FBFEF00EFB103344EA034400FBDE
:1004700006F6A6420AD91CEB040400F1FF3380F013
:100480000081A64240F2FD806444023840EA014007
:10049000A41B00211DB1D4400023C5E90043BDE8E1
:1004A000F0878B4205D90DB1C5E90001002108464E
:1004B000F5E7B3FA83F1002946D1B34202D3824271
:1004C00000F2F580841A66EB030201201746002D26
:1004D000E5D0C5E90047E2E7002A40F09380A1EBB0
:1004E0000C034FEA1C471FFA8CFE0121B3FBF7F601
:1004F00007FB1630230C43EA00430EFB06F098423C
:1005000008D91CEB030306F1FF3802D2984200F22F
:10051000D08046461B1AA4B2B3FBF7F007FB10339A
:1005200044EA03440EFB00FEA64508D91CEB040474
:1005300000F1FF3302D2A64500F2B6801846A4EBC4
:100540000E0440EA0640A5E7C1F120078B4022FADD
:1005500007FC4CEA030C06FA01FE20FA07F426FA1F
:1005600007F344EA0E0400FA01F84FEA1C404FEA90
:100570001449B3FBF0FE1FFA8CF600FB1E3349EA68
:1005800003430EFB06F9994502FA01F20BD91CEB65
:1005900003030EF1FF3A80F08580994540F2828096
:1005A000AEF1020E6344A3EB0909A4B2B9FBF0F368
:1005B00000FB139944EA094403FB06F6A64208D956
:1005C0001CEB040403F1FF3068D2A64266D9023B5B
:1005D000644443EA0E40A41BA0FB02E6B442734607
:1005E000B14652D34FD05DB1B8EB030264EB0904BE
:1005F00004FA07F722FA01F31F43CC40C5E900745F
:1006000000214CE7C2F1200120FA01F30CFA02FCB0
:1006100026FA01F1964033434FEA1C471FFA8CFE3D
:10062000B1FBF7F007FB1016190C41EA064100FB7D
:100630000EF68E4204FA02F408D91CEB010100F117
:10064000FF382DD28E422BD902386144891B9BB2D0
:10065000B1FBF7F607FB161143EA014306FB0EF167
:10066000994208D91CEB030306F1FF3814D29942D2
:1006700012D9023E63445B1A46EA004136E7394626
:10068000EDE6184602E7F045ADD2BEEB020366EB9D
:100690000C060138B146A6E74646ECE7034698E764
:1006A0004046D3E7D6467EE76444023847E708462B
:1006B0000DE7023E63442DE7704700BF2DE9F0418E
:1006C0008AB0002405940694079408940994009431
:1006D0003D4B1A6B42F080021A631A6B02F08002E3
:1006E0000092009A01941A6B42F004021A631A6B8A
:1006F00002F004020192019A02941A6B42F0010284
:100700001A631A6B02F001020292029A03941A6BA6
:1007100042F020021A631A6B02F020020392039A3D
:1007200004941A6B42F002021A631B6B03F002037B
:100730000493049B254D22464FF48041284601F046
:1007400023F801228021284601F01EF80126059693
:100750004FF44413069302230793DFF8788005A92A
:10076000404600F00DFF082305934FF488170697C5
:10077000079605A9404600F003FF4FF40063059378
:100780000697079405A9124800F0FAFE4FF481433A
:10079000059306960794089405A9284600F0F0FEF4
:1007A00022462146062001F067FA062001F074FA7D
:1007B00022462146092001F05FFA092001F06CFA77
:1007C0000AB0BDE8F08100BF0038024000040240DA
:1007D000001402400008024000B583B000210191DE
:1007E000094B1A6B42F480021A631B6B03F48003FB
:1007F0000193019B0A46382001F03EFA382001F0AF
:100800004BFA03B05DF804FB0038024072B6FEE715
:1008100000B585B00023009301930293039316481B
:10082000164A02604FF480324260836003610376AF
:1008300080F820304FF08052C2624FF070628262C6
:10084000C3600123C36180F83030436103F096F93F
:1008500068B903230093012301930023029369469F
:10086000054803F0C5FA20B905B05DF804FBFFF7B1
:10087000CDFFFFF7CBFF00BF2C020020002001407E
:1008800000B595B03022002108A8FFF7FDFC002339
:10089000039304930593069307930193214A116CE4
:1008A00041F080511164126C02F080520192019A61
:1008B00002931D4B1A6842F440421A601B6803F40D
:1008C00040430293029B012308934FF48033099322
:1008D00002230E934FF480020F92082210924FF4DD
:1008E000A872119212930723139308A800F028FB13
:1008F00098B90F23039302230493002305934FF425
:10090000A05306934FF480530793052103A800F0EA
:1009100081FD20B915B05DF804FBFFF777FFFFF705
:1009200075FF00BF0038024000700040000000006A
:10093000F8B501F0EFF9FFF7A3FFFFF7BFFEFFF7F0
:100940004BFFFFF765FF01F02FFA01228021A84835
:1009500000F01AFF3222A749A74803F03BF9A74A43
:1009600000231370D36053609360A54A1370D36063
:100970005360936013E0A34B1B7BDBB2012B40F071
:100980002B81A04B00221A734FF48041984800F04D
:1009900001FF25219C4801F0F3FA0128F9D0974B7B
:1009A0001B78DBB2022BFAD1944B5A68D968B2FBA0
:1009B000F1F29A6001221A7000215960D96098689A
:1009C00089A3D3E90023FFF7B1FC8446CC1704F0D8
:1009D000030220F07043000F40EA011020F0704045
:1009E000034403EB11631344884AA2FB030525F07B
:1009F000030000EB95001B1A24F003042344BCEB16
:100A0000030061EBE3714FF0CC3300FB03F302FB17
:100A10000133A0FB02021A44D30F1B1842F100025B
:100A20005B0843EAC27303EB8303ACEB430C0CF1AA
:100A3000300C754A82F80CC070488168490A744BC2
:100A4000A3FB0131714BC90930315173846871497D
:100A5000A1FB0414A40DA3FB0451C90801EB8101FF
:100A6000A4EB41013031917384686B49A1FB0414FC
:100A7000A40CA3FB0451C90801EB8101A4EB4101C3
:100A80003031D17384686409644FA7FB0414E4090E
:100A9000A3FB0451C90801EB8101A4EB41013031F2
:100AA000117484685E4EA6FB0414640BA3FB04510E
:100AB000C90801EB8101A4EB410130315174846814
:100AC000584DA5FB0414A409A3FB04C1C90801EBFC
:100AD0008101A4EB4101303191748168524CA4FB37
:100AE000011C4FEA5C1CA3FB0CE1C90801EB81016E
:100AF000ACEB41013031D1748168A3FB011C4FEA9A
:100B0000DC0CA3FB0CE1C90801EB8101ACEB41015A
:100B1000303111758068A3FB00C1C90801EB810168
:100B2000A0EB410130315175364801684909A7FBF6
:100B30000171CF09A3FB07C1C90801EB8101A7EB34
:100B40004101303111710168A6FB01614E0BA3FB1D
:100B50000671C90801EB8101A6EB410130315171E9
:100B60000168A5FB01518D09A3FB0561C90801EBD3
:100B70008101A5EB4101303191710168A4FB014174
:100B80004C09A3FB0451C90801EB8101A4EB41010D
:100B90003031D1710468A3FB0414E408A3FB0451B1
:100BA000C90801EB8101A4EB4101303111720168E8
:100BB000A3FB0143DB0803EB8303A1EB43033033C7
:100BC0005372026842F210739A427FF6D4AE00224A
:100BD000026001220273CEE618210B4801F0D0F921
:100BE000DDE600BFAFF3008000E40B54020000001C
:100BF00000040240380100202C020020AC0100203B
:100C0000BC0100209C01002000000020CDCCCCCCF9
:100C1000834B04006BCA5F6B83DE1B43C55A7C0A9F
:100C20005917B7D1D34D62101F85EB51FEE7FEE790
:100C3000FEE7FEE7FEE770477047704708B501F032
:100C400083F808BD08B50C4B1B685B68C3F1320321
:100C50000A4A93609368182B0AD8134601221A7126
:100C6000064A136801331360012000F09DFD08BDA2
:100C7000024B02221A71F3E7CC0100209C010020F4
:100C800008B5044B01221A7300221A60082000F0F4
:100C90008BFD08BD9C01002008B5024800F0AAFEAB
:100CA00008BD00BFCC01002008B5024801F003FEDA
:100CB00008BD00BF7419002008B501228021344806
:100CC00000F062FD334B1B79DBB2022B01D01923FC
:100CD00041E0304B00221A71192307E02E494A687F
:100CE0002E4830F8130002444A600133294A9268C2
:100CF0009A42F3D8274881681939274BDA680A44A1
:100D0000DA605968264A516099689160D968D16063
:100D10000221117000225A60DA609A6001221A7072
:100D2000836807E01C494A681C4830F813000244F5
:100D30004A600133312BF5D9164B9B68C3F132035E
:100D4000154AD3600DE014494A68144830F813007E
:100D500002444A600133312BF5D90F4AD368193365
:100D6000D3600D4BDA6841F287339A420FD90A4BB0
:100D700059680B4A516099689160D968D160022125
:100D8000117000225A60DA609A6001221A7008BD60
:100D9000000402409C010020BC010020380100201A
:100DA000AC01002008B58021274800F0F3FC274B58
:100DB0001B79DBB2012B01D000233DE00023234A45
:100DC000137107E022494A68224830F813000244B0
:100DD0004A6001331D4A92689A42F3D81B498868D9
:100DE0001B4BDA680244DA6058681B4A5060986806
:100DF0009060D868D0600220107000225A60DA60DB
:100E00009A6001221A708B6807E011494A681148FC
:100E100030F8130002444A600133182BF5D90B4B0C
:100E20009A680B4BDA600DE009494A68094830F8C6
:100E3000130002444A600133182BF5D9044AD368E1
:100E40001933D36008BD00BF000402409C0100209C
:100E5000BC01002038010020AC01002082B000213C
:100E600000910B4B5A6C42F480425A645A6C02F463
:100E700080420092009A01911A6C42F080521A64EA
:100E80001B6C03F080530193019B02B0704700BFBD
:100E90000038024030B589B00023039304930593D2
:100EA00006930793026803F1804303F590339A4257
:100EB00001D009B030BD04460025019503F58C33FF
:100EC0005A6C42F480725A645A6C02F48072019235
:100ED000019A02951A6B42F001021A631B6B03F030
:100EE00001030293029B082303930323049303A9A2
:100EF000104800F045FB1048104B036045608560CA
:100F0000C5604FF4806303614FF4006343614FF4A5
:100F1000005383614FF48073C3610562456200F042
:100F2000CDFC18B9044BA3639C63C2E7FFF76EFCCA
:100F3000F8E700BF00000240CC010020106402402E
:100F4000002800F0E08170B582B00446036813F019
:100F5000010F3BD09F4B9B6803F00C03042B2CD05C
:100F60009C4B9B6803F00C03082B21D06368B3F5FE
:100F7000803F4FD0B3F5A02F52D0964B1A6822F481
:100F800080321A601A6822F480221A606368002B8B
:100F900050D000F0E5FE05468E4B1B6813F4003F71
:100FA00014D100F0DDFE401B6428F5D90320B1E127
:100FB000884B5B6813F4800FD8D0864B1B6813F402
:100FC000003F03D06368002B00F09F81236813F07B
:100FD000020F54D07F4B9B6813F00C0F3ED07D4B1B
:100FE0009B6803F00C03082B33D0E368002B68D018
:100FF000794B01221A6000F0B3FE0546754B1B6861
:1010000013F0020F54D100F0ABFE401B0228F5D9BB
:1010100003207FE16F4A136843F480331360B5E720
:101020006C4B1A6842F480221A601A6842F48032CB
:101030001A60ABE700F094FE0546664B1B6813F49C
:10104000003FC3D000F08CFE401B6428F5D903207C
:1010500060E1604B5B6813F4800FC6D15D4B1B6889
:1010600013F0020F03D0E368012B40F05081594A7E
:10107000136823F0F803216943EAC103136023686E
:1010800013F0080F42D063696BB3534B0122C3F8CE
:10109000802E00F065FE05464E4B5B6F13F0020F8D
:1010A00034D100F05DFE401B0228F5D9032031E168
:1010B000484A136823F0F803216943EAC103136027
:1010C000DDE7454B00221A6000F04AFE0546414B21
:1010D0001B6813F0020FD2D000F042FE401B022822
:1010E000F5D9032016E13C4B0022C3F8802E00F016
:1010F00037FE0546374B5B6F13F0020F06D000F04A
:101100002FFE401B0228F5D9032003E1236813F0CA
:10111000040F77D02F4B1B6C13F0805F33D100236B
:1011200001932C4B1A6C42F080521A641B6C03F032
:1011300080530193019B0125284B1B6813F4807F8A
:1011400023D0A368012B34D0052B38D0214B1A6F44
:1011500022F001021A671A6F22F004021A67A368CC
:10116000002B3DD000F0FCFD06461A4B1B6F13F020
:10117000020F46D100F0F4FD801B41F28833984203
:10118000F3D90320C6E00025D6E7144A136843F4D8
:101190008073136000F0E4FD0646104B1B6813F4E7
:1011A000807FCED100F0DCFD801B0228F5D9032022
:1011B000B0E0084A136F43F001031367CFE7054B14
:1011C0001A6F42F004021A671A6F42F001021A679E
:1011D000C5E700BF003802400000474200700040F1
:1011E00000F0BEFD0646524B1B6F13F0020F08D0F5
:1011F00000F0B6FD801B41F288339842F3D90320FA
:1012000088E0EDB9A369002B00F08380484A92681A
:1012100002F00C02082A51D0022B17D0454B0022B5
:101220001A6600F09DFD0446414B1B6813F0007FD9
:1012300042D000F095FD001B0228F5D9032069E09B
:101240003B4A136C23F080531364DBE7394B0022D5
:101250001A6600F085FD0546354B1B6813F0007FCC
:1012600006D000F07DFD401B0228F5D9032051E097
:10127000E369226A1343626A43EA8213A26A52084C
:10128000013A43EA0243E26A43EA0263284A5360AE
:10129000284B01221A6600F063FD0446244B1B68AC
:1012A00013F0007F06D100F05BFD001B0228F5D98A
:1012B00003202FE000202DE000202BE0012B2BD07D
:1012C0001B4B5B6803F48001E269914226D103F075
:1012D0003F02216A8A4223D1616A47F6C0721A40EE
:1012E000B2EB811F1ED103F44031A26A5208013AC9
:1012F000B1EB024F18D103F07063E26AB3EB026FF7
:1013000014D1002006E001207047012002E00120F6
:1013100000E0002002B070BD0120FBE70120F9E7EA
:101320000120F7E70120F5E70120F3E70120F1E7CD
:10133000003802400000474208B5334B9B6803F079
:101340000C03042B5BD0082B5BD12F4B5A6802F0A7
:101350003F025B6813F4800F2CD02B4B5868C0F30E
:1013600088104FEA401CBCEB000C6EEB0E0E4FEAEF
:101370008E1343EA9C634FEA8C11B1EB0C0163EBD3
:101380000E03DB0043EA5173C90011EB000C43F17B
:101390000003590200234FEA4C2041EADC51FFF7D9
:1013A00015F8194B5B68C3F3014301335B00B0FBD5
:1013B000F3F008BD144B5868C0F388104FEA401C86
:1013C000BCEB000C6EEB0E0E4FEA8E1343EA9C63EF
:1013D0004FEA8C11B1EB0C0163EB0E03DB0043EA27
:1013E0005173C90011EB000C43F100039902002373
:1013F0004FEA8C2041EA9C51FEF7E8FFD1E7034811
:10140000D7E70348D5E700BF0038024000127A0052
:101410000024F400002800F09B8070B50D460446BF
:101420004F4B1B6803F00F038B4208D2CBB24C4AE0
:101430001370136803F00F038B4240F08B80236816
:1014400013F0020F17D013F0040F04D0454A93682D
:1014500043F4E0539360236813F0080F04D0414A2B
:10146000936843F4604393603E4A936823F0F0032B
:10147000A1680B439360236813F0010F32D06368B7
:10148000012B21D09A1E012A25D9364A126812F062
:10149000020F61D033498A6822F0030213438B6044
:1014A00000F05EFC06462F4B9B6803F00C0362685D
:1014B000B3EB820F16D000F053FC801B41F288334F
:1014C0009842F0D9032042E0264A126812F4003F05
:1014D000E0D101203BE0234A126812F0007FD9D10D
:1014E000012034E01E4B1B6803F00F03AB4207D909
:1014F000EAB21B4B1A701B6803F00F03AB422DD1ED
:10150000236813F0040F06D0164A936823F4E053BF
:10151000E1680B439360236813F0080F07D0114A6A
:10152000936823F46043216943EAC1039360FFF7A2
:1015300003FF0C4B9B68C3F303130B4AD35CD840E7
:101540000A4B18600A4B186800F0BEFB002070BD03
:10155000012070470120FAE70120F8E70120F6E7B3
:10156000003C024000380240E85000082C000020F7
:1015700028000020014B1868704700BF2C00002095
:1015800000230F2B00F2F68070B582B066E085680C
:101590004FEA430E032404FA0EF425EA0405CC684E
:1015A00004FA0EF42C438460446824EA02044A6876
:1015B000C2F300129A40224342605DE0DC08083426
:1015C00050F8242003F00705AD004FF00F0E0EFA7F
:1015D00005FE22EA0E0E0A69AA4042EA0E0240F80F
:1015E00024205DE0092200E0002202FA0EF22A43E4
:1015F0000234614D45F82420604A94686FEA0C0279
:1016000024EA0C054E6816F4801F01D04CEA04054C
:101610005A4CA560E46802EA04054E6816F4001FFF
:1016200001D04CEA0405554CE560646802EA040503
:101630004E6816F4003F01D04CEA04054F4C65603B
:10164000246822404D6815F4803F01D04CEA040222
:101650004A4C226001330F2B00F28A8001229A400B
:101660000C6804EA020C32EA0404F3D14C6804F07A
:101670000304013C012C8AD94A6802F00302032AC0
:1016800009D0C4685D000322AA4024EA02048A68E3
:10169000AA402243C2604A6802F00302022A8DD0A7
:1016A00004684FEA430E032202FA0EF224EA02040F
:1016B0004A6802F0030202FA0EF2224302604A680C
:1016C00012F4403FC6D0002201922D4A546C44F4DB
:1016D00080445464526C02F480420192019A9C0846
:1016E000A51C254A52F8255003F0030E4FEA8E0E32
:1016F0000F2202FA0EF225EA0205224A90423FF436
:1017000073AF02F58062904222D002F5806290426F
:1017100020D002F5806290421ED002F58062904295
:101720001CD002F5806290421AD002F5806290428D
:1017300018D002F58062904216D002F58062904285
:1017400014D002F5806290423FF44CAF0A224CE77D
:1017500001224AE7022248E7032246E7042244E73F
:10176000052242E7062240E707223EE708223CE73F
:1017700002B070BD704700BF00380140003C01401E
:1017800000380240000002400AB18161704709043C
:1017900081617047436901EA030221EA030141EADA
:1017A000024181617047704708B5054B5B69034290
:1017B00000D108BD024B5861FFF7F5FFF9E700BF04
:1017C000003C014030B405682C6824F480242C606F
:1017D000046863608368402B05D0036899600368E0
:1017E000DA6030BC704703689A600368D960F8E734
:1017F00010B40368D9B210390A4AA2FB0142120997
:10180000094CA25CC2655F2907D96FF30903043351
:101810008365806D5DF8044B70476FF30903836542
:10182000F7E700BFABAAAAAAE0500008836A826962
:1018300092B9012B0AD0022B02D00BB100207047C5
:10184000C36A13F0807F28D100207047C36AB3F1C8
:10185000C07F24D000207047B2F5005F09D0022B72
:1018600025D9032B25D1C36A13F0807F23D1002013
:101870007047032B03D8DFE803F01404140A002098
:101880007047C36A13F0807F0DD100207047C36A90
:10189000B3F1C07F09D000207047012070470120BC
:1018A00070470120704701207047012070470120D8
:1018B00070470020704701207047000070B5044653
:1018C00000F04EFA002C5BD00546022384F8353038
:1018D000002384F834302268136823F00103136076
:1018E00023681A6812F0010F0AD000F039FA431B7E
:1018F000052BF5D920236365032084F8350070BDDE
:101900001A68204911406268A0680243E0680243F7
:101910002069024360690243A0690243E06902430F
:10192000206A02430A43616A04291ED01A602668AD
:10193000756925F00705636A1D43042B07D1A36A67
:101940001D43E36A1BB12046FFF770FF90B9756134
:101950002046FFF74DFFE26D3F2393408360002058
:101960006065012384F83530C9E7E16A206B0143E3
:101970000A43DBE740236365012084F83500BEE7B6
:101980000120BCE73F8010F038B50446856D90F823
:10199000340001282BD0012084F8340094F835005D
:1019A000C0B2012804D0002384F83430022038BDAE
:1019B000022084F83500002060652046FFF702FF12
:1019C000E26D3F239340AB602268136843F0160337
:1019D0001360236C23B12268136843F0080313607B
:1019E0002268136843F0010313600020DFE7022040
:1019F000DDE70000F0B583B0044600230193724B8D
:101A00001D68724BA3FB0535AD0A876D3E68C26D3C
:101A100008239340334210D003681A6812F0040F71
:101A20000BD01A6822F004021A60C26D082393409A
:101A3000BB60436D43F001034365E26D01239340B6
:101A4000334209D02268526912F0800F04D0BB6083
:101A5000636D43F002036365E26D042393403342F8
:101A600009D02268126812F0020F04D0BB60636DC7
:101A700043F004036365E26D10239340334224D0A6
:101A80002268126812F0080F1FD0BB6023681A6822
:101A900012F4802F0DD01B6813F4002F04D1236C97
:101AA0009BB12046984710E0A36C73B1204698473D
:101AB0000BE01A6812F4807F03D11A6822F0080242
:101AC0001A60236C0BB120469847E26D20239340A7
:101AD000334255D02268126812F0100F50D0BB600C
:101AE00094F83530DBB2052B0ED023681A6812F457
:101AF000802F33D01B6813F4002F2AD1636C002B86
:101B00003ED0204698473BE02268136823F0160336
:101B100013602268536923F080035361236CA3B1DF
:101B20002268136823F008031360E26D3F2393409B
:101B3000BB60012384F83530002384F83430236DF2
:101B4000002B3FD0204698473CE0A36C002BE7D108
:101B5000EBE7E36BA3B12046984711E01A6812F453
:101B6000807F09D11A6822F010021A60012384F8DC
:101B70003530002384F83430E36B0BB120469847AE
:101B8000636DFBB1636D13F0010F17D0052384F86B
:101B900035302268136823F001031360019B013381
:101BA0000193AB4204D823681B6813F0010FF5D1F1
:101BB000012384F83530002384F83430E36C0BB112
:101BC0002046984703B0F0BD2C000020B5814E1B85
:101BD000002807DB00F01F02400901239340024A5E
:101BE00042F82030704700BF00E100E0002808DB29
:101BF0000901C9B200F1604000F5614080F80013AE
:101C0000704700F00F000901C9B2014B1954704729
:101C100014ED00E000B500F00700C0F1070CBCF1C6
:101C2000040F28BF4FF0040C031D062B0FD9C31E51
:101C30004FF0FF3E0EFA0CF021EA000199400EFA37
:101C400003FE22EA0E0241EA02005DF804FB0023D3
:101C5000EEE70000074AD36823F4E0631B041B0C83
:101C6000000200F4E060034343F0BF6343F4003339
:101C7000D360704700ED00E010B50446054BD8680E
:101C8000C0F30220FFF7C6FF01462046FFF7AEFF74
:101C900010BD00BF00ED00E008B5FFF799FF08BDDB
:101CA0000138B0F1807F0BD24FF0E0235861054A34
:101CB000F02182F823100020986107221A617047F2
:101CC0000120704700ED00E010B504460E4B1A7875
:101CD0004FF47A73B3FBF2F30C4A1068B0FBF3F0E5
:101CE000FFF7DEFF68B90F2C01D901200AE00022BE
:101CF00021464FF0FF30FFF7BFFF054B1C6000206F
:101D000000E0012010BD00BF260000202C000020B4
:101D10002800002008B50B4B1A6842F400721A60C4
:101D20001A6842F480621A601A6842F480721A607B
:101D30000320FFF78FFF0F20FFF7C6FFFFF78EF896
:101D4000002008BD003C0240034A1168034B1B7889
:101D50000B441360704700BF74020020260000206F
:101D6000014B1868704700BF7402002038B5044664
:101D7000FFF7F6FF0546B4F1FF3F02D0044B1B7896
:101D80001C44FFF7EDFF401BA042FAD338BD00BF53
:101D900026000020034AD2F8883043F47003C2F8CA
:101DA0008830704700ED00E008B500220F49104868
:101DB00002F0F4F870B90F490D4802F006F960B965
:101DC0000D490B4803F0FAF850B9094802F017F929
:101DD00048B908BDFEF71AFDEDE7FEF717FDEFE77E
:101DE000FEF714FDF1E7FEF711FDF2E764000020B5
:101DF00078020020D80000208000002012230B80F1
:101E0000004870475000002004230B8000487047B2
:101E10004C000020002393421ED200B510E00CF1CC
:101E2000370C01F813C000014FEA430C0CF1010C10
:101E30004FF0000E01F80CE00133DBB2934209D2FF
:101E40004FEA107CB0F1204FE9D20CF1300C01F8D0
:101E500013C0E8E75DF804FB7047000038B50B4B92
:101E6000D3F8100AD3F8144AD3F8183AC01800D19E
:101E700038BD074D08222946FFF7CCFF042205F1A3
:101E800010012046FFF7C6FFF2E700BF0070FF1FFA
:101E90003200002008B51A230B80FFF7DFFF01484E
:101EA00008BD00BF3000002008B50A4628B9054922
:101EB000054802F0F9FD034808BD0249024802F056
:101EC000F3FDF8E754050020F850000810B50A4665
:101ED000034C2146034802F0E7FD204610BD00BF39
:101EE000540500201051000808B50A4628B90549D4
:101EF000054802F0D9FD034808BD0249024802F036
:101F0000D3FDF8E7540500202451000808B50A461F
:101F100028B90549054802F0C7FD034808BD024934
:101F2000024802F0C1FDF8E75405002030510008D6
:101F300000207047002070470020704710B5014610
:101F4000044C204603F053F8204603F077F80020B5
:101F500010BD00BF7802002010B5064C00220649D3
:101F6000204603F036F80549204603F040F80020EB
:101F700010BD00BF7802002054070020540F00203D
:101F8000094BD3F8BC32D3F814320BB1012070479F
:101F900010B5054C0A460146204603F01AF82046C3
:101FA00003F031F810BD00BF7802002030B589B0D1
:101FB0000023039304930593069307930368B3F1F7
:101FC000A04F01D009B030BD00250195164C236B00
:101FD00043F001032363236B03F001030193019B8F
:101FE0004FF4C053039302230493032306930A235D
:101FF000079303A90D48FFF7C3FA636B43F080030F
:1020000063630295636C43F480436364636C03F41D
:1020100080430293029B2A4629464320FFF72CFE69
:102020004320FFF739FECDE70038024000000240B0
:1020300008B500F29C41D0F8E00401F0F6FF08BDBD
:1020400008B501EBC10300EB8303D3F86022D0F89D
:10205000E00402F0BDF808BD08B501EBC10300EBD8
:1020600083031A6AD0F8E00402F017F908BD08B536
:10207000D0F8E00402F057F808BD10B50446C17965
:1020800011B1022909D10121D4F8E00402F02CF8A1
:10209000D4F8E00401F0F5FF10BDFEF7B7FB012115
:1020A000F2E7000010B50446D0F8E00402F01FF893
:1020B0002268D2F8003E43F00103C2F8003EE37A02
:1020C00023B1034A136943F00603136110BD00BF37
:1020D00000ED00E008B5D0F8E00402F017F808BD04
:1020E00008B5D0F8E00402F046F808BD08B5D0F80D
:1020F000E00402F029F808BD08B5D0F8E00402F0C9
:1021000051F808BD08B5D0F8E00402F04DF808BD5C
:1021100002780AB10020704710B503461548C0F890
:10212000E034C3F8C8024FF0A043036004230371F6
:102130000222C2710023837142728372C3720373DD
:102140008373C37300F0EEF880B90A4C80212046F7
:1021500000F0B6FE40220021204600F08BFE8022D7
:102160000121204600F086FE002010BDFEF74EFB48
:10217000EBE700BF74190020D0F8C83211F0800FCF
:1021800008D101F07F0101EBC10103EB810393F85A
:102190005602704701F07F0101EBC10103EB81039F
:1021A000987D704708B5D0F8C80200F0BFFA08BDA6
:1021B00000487047541700207047032805D8DFE80F
:1021C00000F005040205012070470320704708B5A0
:1021D000D0F8C80200F027F9FFF7EFFF08BD08B5F7
:1021E00094461A466346D0F8C80200F0FCF9FFF79F
:1021F000E4FF08BD08B5D0F8C80200F03AFAFFF7CE
:10220000DCFF08BD08B5D0F8C80200F0BDFAFFF742
:10221000D4FF08BD08B5D0F8C80200F0F8FAFFF7FF
:10222000CCFF08BD08B5D0F8C80200F0C9F9FFF727
:10223000C4FF08BD08B5D0F8C80200F080FAFFF767
:10224000BCFF08BD08B5D0F8C80200F04AFAFFF795
:10225000B4FF08BD2DE9F04383B0D0F8008001EB56
:10226000C10300EB83039A6A5B6A9A4254D807461B
:102270000C469B1A01EBC10200EB8202D2699A4222
:1022800000D31A4602F103094FEA990915E006F155
:1022900003094FEA9909BB7904EBC40507EB8505EF
:1022A000296A0093B3B2E2B2404601F048F92B6AC2
:1022B00033442B62AB6A3344AB6208EB441303F53F
:1022C00010639B699BB24B4512D304EBC40307EB2D
:1022D00083039A6A5B6A9A420AD24BB19B1A04EB57
:1022E000C40207EB8202D6699E42D0D31E46CEE7D7
:1022F00004EBC40307EB83077A6ABB6A9A420FD8E0
:1023000004F00F040122A240D8F8343823EA020373
:10231000C8F83438002000E0012003B0BDE8F083A5
:102320000020FAE730B583B000287AD0044605686B
:1023300090F89534C3B1032384F89534B5F1A04FD8
:1023400017D0206800F0AEFE237C8DF80030231DEE
:102350000ECB206800F0E5FD70B1022384F89534BF
:102360000125284603B030BD80F89434FFF71EFEE7
:10237000E1E70023A371E4E70021206801F0F5FA0A
:10238000024608B9034617E0022384F89534012574
:10239000E7E703EBC30104EB8101012048750B75EE
:1023A000CB8500200876C861086203EBC30104EB0B
:1023B000810148620133DBB220799842E9D816E006
:1023C00002EBC20304EB8303002183F8551283F868
:1023D000542283F85812C3F85C12C3F8601202EB5F
:1023E000C20304EB8303C3F864120132D2B29042F9
:1023F000E6D8237C8DF80030231D0ECB206800F03A
:10240000A7FE054620B1022384F895340125A8E7EC
:1024100000236374012384F89534206801F064FA82
:102420009FE701259DE7036890F89424012A1AD0BC
:1024300010B50446012280F89424DA6812F0400FA7
:1024400002D0427B012A09D0206800F025FE2068D6
:1024500001F03CFA002084F8940410BD9A6B42F419
:1024600080329A63F0E702207047000070B504469E
:102470000D460068066C00EB411303F530639A6863
:10248000A179012911D038498E4256D03DB905EBCA
:10249000C50304EB8303D3F86432002B5ED0E9B2AA
:1024A0002046FFF7CDFD002070BD12F0080F09D0C7
:1024B0002E498E42F7D912F4004FF4D04FF4004267
:1024C0009A60F0E712F0200F02D020229A60EAE72B
:1024D00012F0280FE7D125498E4206D912F4004F99
:1024E00003D04FF400429A60DDE705EBC50204EB30
:1024F0008202D2F874121B69C3F31203CB1AC2F81A
:1025000068327DB905EBC50204EB8202D2F8642281
:102510006AB105EBC50204EB8202D2F860121944DD
:10252000C2F86012E9B22046FFF78AFDBBE704F269
:102530009C42012101F058FAF4E712F4004F03D055
:102540004FF400429A60AEE712F0200F01D0202233
:102550009A60E9B22046FFF773FDA4E704F29C42BB
:10256000002101F041FA9AE70A31544F0A30544FE2
:1025700038B5044603681D6C03EB4113D3F8081B00
:102580000E4A954207D903F5306311F4004F02D08B
:102590004FF400429A602046FFF74AFD074B9D42E8
:1025A00002D9A379012B01D0002038BD04F29C424E
:1025B0000121206801F018FAF6E700BF0A30544FF5
:1025C00090F89434012B0CD010B50446012380F808
:1025D00094344174006801F069F9002084F894048F
:1025E00010BD0220704738B505468C4611F0800FAB
:1025F0002BD101F00F0E0EEBCE04A40004F51474E1
:102600000444211D0EEBCE0E00EB8E0E00208EF842
:1026100055020CF00F0C81F800C0C2F30A028A6068
:102620000B714A780AB1A1F81AC0022B1CD095F898
:102630009434012B1BD0012385F89434286800F0D2
:1026400062FE002085F8940438BD01F00F0000EB15
:10265000C001890010312944043100EBC00005EBB2
:10266000800001244475D4E700234B71DFE702208A
:10267000EAE710B504460A4611F0800F20D101F0B8
:102680000F0000EBC0039B0003F514732344191DD6
:1026900000EBC00004EB8000002380F8553202F00C
:1026A0000F020A7094F89434012B18D0012384F897
:1026B0009434206800F074FE002084F8940410BD67
:1026C00001F00F0000EBC0039B0010332344191DE1
:1026D00000EBC00004EB800001234375DFE702201C
:1026E000EDE710B5144601F00F0C0CEBCC0189009E
:1026F00001F51471014404310CEBCC0E00EB8E0E8D
:10270000CEF86022CEF864320023CEF868328EF81C
:1027100055328EF854C28279012A04D0006800F044
:1027200025FF002010BDCEF87042F7E701F00F0141
:1027300001EBC10100EB8100D0F86802704710B5D1
:10274000144601F00F0C0CEBCC0189001031014450
:1027500004310CEBCC0E00EB8E0ECEF82020CEF820
:1027600024300023CEF8283001238EF815308EF85F
:1027700014C082799A4204D0006800F0F7FE00206D
:1027800010BDCEF83040F7E738B501F00F050279FB
:10279000AA4238D304460B4611F0800F1FD101EB3B
:1027A000C101890001F514710144043103EBC30335
:1027B00000EB8303002283F8552201238B700D70F8
:1027C00094F89434012B20D0012384F894342068A9
:1027D00001F011F885B1002084F8940438BD05EBB0
:1027E000C501890010310144043105EBC50300EB3C
:1027F000830301225A75E0E704F29C42A179206824
:1028000001F0F2F8E7E70120E8E70220E6E701F04F
:102810000F0302799A4230D310B5044611F0800FAD
:102820001ED103EBC301890001F514710144043189
:1028300003EBC30200EB8202002082F85502002263
:102840008A700B7094F89434012B18D0012384F80B
:102850009434206800F0FCFF002084F8940410BD3C
:1028600003EBC301890010310144043103EBC302BF
:1028700000EB820201205075E1E701207047022041
:10288000EDE708B511F0800F0CD101F00F0101EB5D
:10289000C101890001F5147101440431006800F0A0
:1028A000EFFD08BD01F00F0101EBC10189001031FE
:1028B00001440431F2E72DE9F04F83B00446056886
:1028C000284601F04EF810B103B0BDE8F08F06467F
:1028D000206801F017F80028F6D005F50067BB68FE
:1028E000C3F30D23C4F8D434206801F00BF810F0C2
:1028F000020F04D02268536903F002035361206879
:1029000001F000F810F0100F15D02268936923F041
:1029100010039361D5F8208008F00F0908F4F01334
:10292000B3F5802F4CD0B3F5402F6FD02268936958
:1029300043F010039361206800F0E4FF10F4002FCF
:1029400076D1206800F0DEFF10F4802F40F0E080A8
:10295000206800F0D7FF0028C0F26181206800F0F5
:10296000D1FF10F4006F09D0BB6813F0010F40F0E5
:102970006E812268536903F400635361206800F09C
:10298000C1FF10F4805F40F06681206800F0BAFF5C
:1029900010F4005F40F0B381206800F0B3FF10F046
:1029A000080F40F0C481206800F0ACFF10F0800FE9
:1029B00000F0D781AB6923F08003AB610126C0E151
:1029C00047F6F07318EA030FB0D04FEA181A4FEA2F
:1029D000C903019309EBC90B04EB8B0BC8F30A1273
:1029E000DBF86012284600F0E3FEDBF86032CAF341
:1029F0000A0A5344CBF86032DBF86832019A4A4441
:102A000004EB82025344C2F868328FE7082204F2D2
:102A10009C41284600F0CCFE09EBC90304EB83037C
:102A2000D3F86822C8F30A184244C3F868227DE745
:102A3000206800F06BFF8046B14635E005EB491396
:102A40000122C3F8082B49462046FFF70FFD3CE062
:102A500005EB49130822C3F8082B49462046FFF727
:102A600087FD35E009EBC90304EB830393F8573284
:102A7000012B41D005EB49130222C3F8082B1AF0B1
:102A8000200F04D005EB49132022C3F8082B1AF4B9
:102A9000005F05D005EB49134FF40052C3F8082B33
:102AA00009F101094FEA5808B8F1000F3FF449AFA6
:102AB00018F0010FF4D05FFA89FB5946206800F046
:102AC00035FF824610F0010FB8D11AF0080FBFD1C0
:102AD0001AF0100F04D005EB49131022C3F8082B8D
:102AE0001AF0020FCBD06B6913F0800FBAD07B685D
:102AF00043F480637B60B5E709EBC90304EB830310
:102B0000002283F8572259462046FFF7E9FAB1E739
:102B1000206800F003FF8046B14625E05946204674
:102B2000FFF79AFA1AF0080F04D005EB49130822B0
:102B3000C3F808291AF0100F04D005EB491310222E
:102B4000C3F808291AF0400F04D005EB49134022BE
:102B5000C3F808291AF0020F40D11AF0800F59D19A
:102B600009F101094FEA5808B8F1000F3FF4F0AE3F
:102B700018F0010FF4D05FFA89FB5946206800F085
:102B8000DEFE824610F0010FCCD009F00F020121C9
:102B900001FA02F27B6B23EA02037B6305EB491324
:102BA000C3F80819A3798B42B8D109EBC90304EB28
:102BB00083031A6AD9690A441A62B9F1000FADD1C8
:102BC00009EBC90304EB83035B6A002BA6D104F273
:102BD0009C420121206800F007FF9FE749462846F4
:102BE00000F066FA09EBC90304EB8303DB7D012BDC
:102BF00005D005EB49130222C3F80829ADE709EB1C
:102C0000C90304EB83030022DA7559462046FFF717
:102C10006DFAEEE749462046FFF71CFBA0E77B680C
:102C200023F001037B6094F8CC34012B08D02046BC
:102C3000FFF750FA2268536903F0004353618DE6B1
:102C4000002184F8CC14204600F03EF9F2E720463B
:102C5000FFF728FA8DE67B6823F001037B601021E3
:102C6000206800F025FA1AE005EB46134FF67F3195
:102C7000C3F80819D3F8002922F40012C3F8002978
:102C8000C3F8081BD3F8002B22F40012C3F8002B62
:102C9000D3F8002B42F00062C3F8002B01362379F1
:102CA000B342E1D8FB6943F00113FB61E37BDBB185
:102CB000D7F8843043F00B03C7F884307B6C43F0C3
:102CC0000B037B64D5F8003823F4FE63C5F80038A5
:102CD00004F29C42A179206800F086FE22685369C4
:102CE00003F48053536150E67B6943F4005343F08F
:102CF0002B037B613B6943F00B033B61E2E72068F8
:102D000000F064FE206800F0EDFAE0712668FEF73E
:102D100031FC0146E279304600F04CF92046FFF7DD
:102D2000ACF92268536903F40053536134E620463A
:102D3000FFF79DF92268536903F00803536132E6F7
:102D400001362379B3420CD906EBC60304EB8303A7
:102D500093F85732012BF3D1F1B22046FFF791FDE2
:102D6000EEE7206800F0CEFD10F4801F25D120682A
:102D700000F0C8FD10F4001F58D0012326E00136F2
:102D80002379B3421BD905EB4613D3F8002906EB90
:102D9000C60304EB83031B7E012BF0D1002AEEDA7D
:102DA00006EBC60304EB83030122DA7566F07F01AC
:102DB000C9B22046FFF765FDE1E70126E0E722689A
:102DC000536903F480135361D1E7013322799A42A6
:102DD00027D905EB4312D2F8001B03EBC30204EB27
:102DE000820292F85822012AEFD10029EDDAD4F8B4
:102DF000D42482EA114212F0010FE6D103EBC302A0
:102E000004EB8202012182F85712AA6942F0800283
:102E1000AA616A6912F0800FD7D17B6843F400730E
:102E20007B602268536903F400135361206800F04B
:102E300069FD10F0804F10D1206800F063FD10F0A4
:102E4000040F3FF441AD23685D6815F0040F0DD108
:102E5000226853682B43536036E52046FFF74CF950
:102E60002268536903F080435361E5E72046FFF78A
:102E700049F9EDE710B40468606A31B940EA0240EC
:102E8000A06200205DF8044B70478C46A36A00EBFB
:102E90001340002308E003F1400104EB810149687D
:102EA00000EB11400133DBB20CF1FF318B42F2D366
:102EB00040EA02400CF13F0104EB81046060E0E76E
:102EC0000368596200207047704782B00023019365
:102ED000019B01330193019BB3F1706F1CD803690F
:102EE000002BF5DA0A23019302E0019B013B0193D9
:102EF000019B002BF9D1036943F001030361019B9E
:102F000001330193019BB3F1706F08D8036913F08B
:102F1000010FF4D1002000E0032002B0704703202D
:102F2000FBE784B010B5044603A880E80E009DF8C6
:102F30001130012B21D1A36B23F48033A363E36809
:102F400023F4840323F04003E360E36823F4401395
:102F5000E3609DF81830012B0AD02046FFF7B5FF3B
:102F60009DF80E30012B1CD0BDE8104004B0704716
:102F7000E36843F48013E360EFE7E36843F0400362
:102F8000E3602046FFF7A1FF9DF8153023B9A36B3E
:102F900043F48033A363E3E7A36B23F48033A36399
:102FA000DEE7A36843F00603A360A36843F02003B1
:102FB000A360D9E7022A0AD00922C36823F4705318
:102FC000C360C36843EA8223C36000207047234B79
:102FD0000B44234A93422FD9224B0B44224A93425B
:102FE0002CD9A1F57403A3F51053204A934227D995
:102FF000A1F18373A3F5E7431D4A934222D31D4BEE
:103000000B441D4A93421FD91C4B0B441C4A93424C
:103010001CD31C4B0B441C4A934219D3A1F1B77328
:10302000A3F55853194A934214D3194B0B44194A28
:10303000934211D20722C0E70F22BEE70E22BCE75F
:103040000D22BAE70C22B8E70B22B6E70A22B4E752
:103050000922B2E70822B0E70622AEE7405327FF75
:10306000FF340C00401E1BFF3F420F007F4F120039
:1030700020D6130060B6E5FE5FE3160000D3CEFE57
:1030800040771B00C05BB3FEC09121002075380063
:10309000E05459FEE09C4100836843F001038360E3
:1030A00000207047836823F001038360002070478D
:1030B00082B000230193019B01330193019BB3F183
:1030C000706F15D80369002BF5DA0023019389018D
:1030D00041F020010161019B01330193019BB3F198
:1030E000706F08D8036913F0200FF4D1002000E0BE
:1030F000032002B070470320FBE782B00023019356
:10310000019B01330193019BB3F1706F13D80369E5
:10311000002BF5DA0023019310230361019B013397
:103120000193019BB3F1706F08D8036913F0100F7E
:10313000F4D1002000E0032002B070470320FBE739
:10314000D0F800381943C0F800180020704700007C
:1031500084B0F8B5044607A880E80E00002306E016
:1031600003F1400204EB82020021516001330E2B77
:10317000F6D99DF8266006BBD4F8043843F0020364
:10318000C4F80438A36B43F40013A363A36B23F4C4
:103190000023A363A36B23F48023A3630023C4F859
:1031A000003E9DF82130012B15D19DF81F306BB9E1
:1031B00000212046FFF7C4FF11E0A36B23F40013A6
:1031C000A363A36B43F40023A363E7E70121204635
:1031D000FFF7B6FF03E003212046FFF7B1FF102100
:1031E0002046FFF765FF054600B101252046FFF7A1
:1031F00084FF00B1012504F5006C0023CCF81030E9
:10320000CCF81430CCF81C300AE0CBB94FF0006099
:10321000C2F8000900220A614FF67F328A6001334A
:103220009DF81C10994210D904EB431202F510616D
:10323000D2F800090028E8DB0020C2F80009E9E71D
:103240004FF09040C2F80009E4E700230AE0BBB168
:103250004FF09047C2F8007B002202614FF67F32A8
:1032600082600133994210D904EB431202F53060B9
:10327000D2F8007B002FEADB0027C2F8007BEBE7E7
:103280004FF00067C2F8007BE6E7DCF8103023F46B
:103290008073CCF810300023A3616FF0804363612A
:1032A0009DF81E301BB9A36943F01003A361A26906
:1032B0000B4B1343A3619DF822301BB1A36943F06C
:1032C0000803A361012E04D02846BDE8F84004B0ED
:1032D0007047A36943F0804343F00403A361F3E71D
:1032E00000383C80D0F8083803F00603022B04D0E5
:1032F000062B04D02BB90020704702207047022013
:1033000070470F20704710B591F800C04B78012B23
:1033100023D000F5006ED0F81C380CF00F04012209
:10332000A24043EA0243C0F81C3800EB4C10D0F82E
:10333000003B13F4004F0ED1D0F8003B8A68C2F373
:103340000A02097942EA8142134343F0805343F46D
:103350000043C0F8003B002010BDD0F81C280CF042
:103360000F0E03FA0EF39BB21343C0F81C3800EBA8
:103370004C10D0F8003913F4004FECD1D0F80039DC
:103380008A68C2F30A02097942EA814242EA8C520F
:10339000134343F0805343F40043C0F80039DAE7A5
:1033A00030B40B784A78012A26D000EB4313D3F8C7
:1033B000002B002A52DBD0F83C480A7802F00F02BA
:1033C0004FF0010C0CFA02F224EA0242C0F83C2849
:1033D000D0F81C28097801F00F010CFA01FC22EA50
:1033E0000C42C0F81C28D3F8001B234A0A40C3F83B
:1033F000002B002030BC704700EB4313D3F80029AA
:10340000002A1EDBD0F83C580A7802F00F02012493
:1034100004FA02F292B225EA0202C0F83C28D0F87F
:103420001C28097801F00F018C40A4B222EA0402A2
:10343000C0F81C28D3F80019104A0A40C3F8002924
:10344000D7E7D3F8002942F00062C3F80029D3F887
:10345000002942F08042C3F80029D3E7D3F8002BBB
:1034600042F00062C3F8002BD3F8002B42F08042F8
:10347000C3F8002B9FE700BF0078F3EF007833EC30
:1034800010B483B0024600230193487801280BD082
:103490000B7802EB4313D3F8000B00282DDB002040
:1034A00003B05DF8044B70470B7802EB4313D3F87D
:1034B0000049002C01DB0020F2E7D3F8004944F07A
:1034C0000064C3F800490B7802EB4313D3F80049BA
:1034D00044F08044C3F80049019B01330193019CEF
:1034E00042F210739C42DBD80B7802EB4313D3F803
:1034F0000039002BF0DB0020D2E7D3F8000B40F0BE
:103500000060C3F8000B0B7802EB4313D3F8000BF9
:1035100040F08040C3F8000B019B013301930198F8
:1035200042F21073984208D80B7802EB4313D3F899
:10353000003B002BF0DB0020B2E70120B0E710B524
:103540009DF8084084B903334FEA930E4FF0000C06
:1035500008E000EB023303F5805351F8044B1C6084
:103560000CF1010CF445F4D3002010BDF0B583B08C
:103570000C784B78012B2DD000EB441C0CF53063FC
:103580001D696FF312051D611D696FF3DC451D6137
:10359000002C40F0CE800C690CB18C680C618C68FA
:1035A0000C621D69C4F312042C431C611C6944F4B1
:1035B00000241C61012A00F0DF800B79012B00F050
:1035C000E180DCF8003B43F00443CCF8003B0020F2
:1035D00003B0F0BD0B6973BB00EB4413D3F8105973
:1035E0006FF3DC45C3F81059D3F8105945F40025A2
:1035F000C3F81059D3F810596FF31205C3F81059D6
:10360000012A54D000EB4414D4F8003943F00443A9
:10361000C4F800390B79012B72D00B69002BD6D07E
:10362000D0F83438097801F00F0101228A401343A1
:10363000C0F83438CBE700EB441303F510631D6981
:103640006FF312051D611D696FF3DC451D6184B9BF
:103650000E698D68AE4200D90D611D6945F40025E3
:103660001D611D690E69C6F3120C45EA0C051D614A
:10367000C6E70D698E683544013DB5FBF6F51E6958
:103680001FFA85FC494F07EAC54535431D610D7991
:10369000012DE6D11D6925F0C0451D611D694FEA68
:1036A0004C7C0CF0C04C45EA0C051D61D9E7CB6998
:1036B0001BB100EB4412C2F814390B79012B08D06E
:1036C00000EB4414D4F8003943F00443C4F8003943
:1036D0007DE7D0F8083813F4807F08D100EB44125E
:1036E000D2F8003943F00053C2F80039E8E700EBA4
:1036F0004412D2F8003943F08053C2F80039DFE7B2
:10370000D0F8083813F4807F0CD1D4F8003943F096
:103710000053C4F8003900920B8A0A78C968FFF791
:103720000EFF54E7D4F8003943F08053C4F8003951
:10373000F1E70C6954B91C698D68C5F312052C4377
:103740001C611C6944F400241C6133E78D682C441F
:10375000013CB4FBF5F4A4B204FB05F50D621D6950
:10376000124E06EAC4442C431C611C690D6AC5F361
:1037700012052C431C611DE7CA68002A3FF41DAFE7
:103780005A611AE7D0F8083813F4807F06D1DCF8C4
:10379000003B43F00053CCF8003B12E7DCF8003B61
:1037A00043F08053CCF8003B0BE700BF0000F81F4C
:1037B00010B5844608464FEA920E02F00302002339
:1037C00005E00CF58051096840F8041B013373458E
:1037D000F7D37AB10CF5805CDCF800400021CBB265
:1037E000DB0024FA03F300F8013B0131013A92B205
:1037F000002AF4D110BD0B784A78012A14D000EBCE
:103800004310D0F8002B002A06DB2BB1D0F8003B88
:1038100023F08043C0F8003BD0F8003B43F4001392
:10382000C0F8003B0020704700EB4310D0F800299F
:10383000002A06DB2BB1D0F8003923F08043C0F812
:103840000039D0F8003943F40013C0F80039E9E733
:103850000B784A78012A0ED000EB4310D0F8003BD9
:1038600023F40013C0F8003B0B79023BDBB2012BC1
:1038700015D90020704700EB4310D0F8003923F42D
:103880000013C0F800390B79023BDBB2012BF0D8F2
:10389000D0F8003943F08053C0F80039E9E7D0F898
:1038A000003B43F08053C0F8003BE2E7D0F800381B
:1038B00023F4FE63C0F80038D0F80038090101F4A1
:1038C000FE610B43C0F8003800207047D0F8003E7E
:1038D00023F00303C0F8003ED0F8043823F00203BD
:1038E000C0F8043800207047D0F8003E23F00303EE
:1038F000C0F8003ED0F8043843F00203C0F80438A2
:10390000002070474269806910407047D0F818382D
:1039100000F50060C0691840000C7047D0F81838F6
:1039200000F50060C069184080B2704700EB41119B
:10393000D1F8082B00F50060406910407047D0F8BE
:103940001028D0F8343801F00F0C23FA0CF3DB0107
:10395000DBB2134300EB411000F5106080681840A3
:103960007047406900F00100704738B50546C368EC
:1039700023F0C043C360012913D019BBC36843F0CF
:103980008043C36000240A20FEF7F0F90A34284679
:10399000FFF7E7FF08B1C72CF5D9C82C14D00020D9
:1039A00038BDC36843F00053C36000240A20FEF70B
:1039B000DDF90A342846FFF7D4FF0128EDD0C72CE3
:1039C000F4D9EAE70120EBE70120E9E7D0F8003974
:1039D0006FF30A03C0F80039D0F8043843F4807359
:1039E000C0F804380020704710B4046C154B9C429A
:1039F00003D9D0F8003B002B16DB0024C0F8104B95
:103A0000D0F8104B44F40024C0F8104BD0F8104B01
:103A100044F01804C0F8104BD0F8104B44F0C044E8
:103A2000C0F8104B012903D000205DF8044B70470B
:103A3000C0F8142BD0F8003B43F08023C0F8003BC3
:103A4000F2E700BF0A30544F4A4B5A6822F4403222
:103A50005A605A6841680A435A600268536823F4FE
:103A60008073536002685368016943EA012353601D
:103A70000268536823F0407353600268536881689A
:103A80000B4353600268936823F4006393600268F9
:103A90009368C1680B439360826A374B9A4257D050
:103AA0000268936823F07063936002689368816A88
:103AB0000B4393600268936823F04053936002685D
:103AC0009368C16A0B4393600268936823F0020312
:103AD000936002689368017E43EA4103936090F823
:103AE0002030002B3FD00268536843F400635360DA
:103AF0000268536823F46043536001684B68426A6C
:103B0000013A43EA42334B600268D36A23F47003FC
:103B1000D3620168CB6AC269013A43EA0253CB62BD
:103B20000268936823F4007393600268936890F8C6
:103B3000301043EA412393600268936823F4806362
:103B4000936002689368416943EA812393607047F8
:103B50000268936823F0706393600268936823F0AF
:103B600040539360B0E70268536823F400635360E6
:103B7000CAE700BF002301400100000F38B310B5B1
:103B80000446036C43B1236C13F0100F0BD00120DB
:103B9000002384F83C3010BDFDF77CF900236364FA
:103BA00084F83C30EFE7236C23F4885323F00203BE
:103BB00043F0020323642046FFF746FF00206064C1
:103BC000236C23F0030343F001032364E0E70120A7
:103BD0007047000010B582B013460022019290F8A1
:103BE0003C20012A00F0A7800446012280F83C20F6
:103BF0000268906810F0010F13D1906840F0010046
:103C000090604E4A10684E4AA2FB0020800C00EBE8
:103C10004000019002E001980138019001980028CD
:103C2000F9D12268906810F4807F03D0906820F466
:103C3000807090602268906810F0010F70D0206C46
:103C400020F4E06020F0010040F4807020645268AD
:103C500012F4806F05D0226C22F4405242F480525C
:103C60002264226C12F4805F3BD0626C22F0060268
:103C70006264002284F83C20A26B3248D063A26BBD
:103C800031481064A26B3148D06422686FF0220082
:103C900010602068426842F080624260206882685A
:103CA00042F48072826020680A4600F14C01A06BE9
:103CB000FDF76AFE264B5B6813F01F0F23D12368C4
:103CC000244A934216D002F5807293420CD0224AC5
:103CD00093422ED102F58072526812F0100F28D153
:103CE00008E000226264C4E702F50072526812F034
:103CF0001F0FECD19A6812F0405F1AD19A6842F017
:103D000080429A6015E02368124A934211D19A6862
:103D100012F0405F0DD19A6842F080429A6008E04C
:103D2000236C43F010032364636C43F0010363646A
:103D3000002002B010BD0220FBE700BF2C000020D5
:103D400083DE1B437F3D00085D3D0008693D0008A0
:103D500000230140002001400022014008B5806B93
:103D6000FDF720F808BD704708B5806B4023036459
:103D7000436C43F004034364FFF7F5FF08BD08B547
:103D80000346806B026C12F0500F25D1036C43F494
:103D90000073036403689A6812F0405F19D1027ED1
:103DA000BAB9DA6A12F4700F03D09A6812F4806F0D
:103DB0000FD15A6822F020025A60036C23F48073FA
:103DC0000364036C13F4805F03D1036C43F00103BD
:103DD0000364FCF771FF08BD026C12F0100F04D1F0
:103DE000826BD26C18469047F5E7FFF7BCFFF2E70D
:103DF00030B482B00022019290F83C20012A00F0F9
:103E0000C0800346012280F83C200A68092A40D974
:103E10000468E06892B202EB42021E3A4FF0070CCF
:103E20000CFA02F220EA0202E2601C68E0680A88EA
:103E300002EB42021E3A8D6805FA02F20243E2608A
:103E40004A68062A3CD81C68606B02EB8202053A7D
:103E50004FF01F0C0CFA02F220EA020262631C68A7
:103E6000606B4A6802EB8202053AB1F800C00CFAB6
:103E700002F2024362631868434A904250D01868C5
:103E8000414A904259D0002083F83C0002B030BC37
:103E900070470468206992B202EB42024FF0070CAF
:103EA0000CFA02F220EA020222611C6820690A88E8
:103EB00002EB42028D6805FA02F202432261BFE77B
:103EC0000C2A16D81D68286B02EB8202233A1F24A5
:103ED00004FA02F220EA02022A631D68286B4A688B
:103EE00002EB8202233A0C8804FA02F202432A63AC
:103EF000C1E71D68E86A02EB8202413A1F2404FA16
:103F000002F220EA0202EA621D68E86A4A6802EBED
:103F10008202413A0C8804FA02F20243EA62AAE7FA
:103F20000A68122AABD1194A506820F40000506088
:103F3000506840F480005060A1E70A68144882424B
:103F400001D0112A9FD1114A506820F4800050609E
:103F5000506840F40000506009680D4A914292D1C7
:103F60000C4A12680C49A1FB0212920C02EB82026D
:103F700052000192019A002A85D0019A013A0192D9
:103F8000F8E7022082E700BF002001400023014043
:103F9000120000102C00002083DE1B4398B108B5EE
:103FA00003460020C3F8B802C3F8C402C3F8D00225
:103FB00009B1C3F8B412012183F89C121A70184693
:103FC000FEF7A6F808BD0320704710B582B00023A5
:103FD000ADF8063089B10446C0F8B812CB6A23B1F7
:103FE0000DF106009847C4F8D002D4F8D832013356
:103FF000C4F8D832002002B010BD0320FBE708B59A
:10400000FEF7E5F808BD08B5D0F8B83213B11B6863
:10401000984708BD0020FCE708B5D0F8B8325B68C7
:10402000984700B908BD0320FCE738B5044600F204
:10403000AA25284600F0CDF90123C4F89432B4F83B
:10404000B032C4F8983294F8AA1201F01F03012B81
:1040500007D0022B0AD073B92946204600F08EFB08
:1040600038BD2946204600F0C4FBF9E72946204622
:1040700000F001FCF4E701F080012046FEF7C2F8F1
:10408000EEE7F8B50446012380F89C320023C0F81F
:1040900094324360C0F8A43280F8A032D0F8B8322D
:1040A000E3B15B68E3B1002198470746D0B94023EC
:1040B000002211462046FEF792F8012684F863613B
:1040C0004025A4F860512B46002280212046FEF7AF
:1040D00086F884F8236025843846F8BD0027E6E793
:1040E0000027E4E70327E2E701740020704790F817
:1040F0009C32DBB2042B04D090F89C32DBB280F807
:104100009D32042380F89C320020704790F89C3246
:10411000DBB2042B01D00020704790F89D32DBB257
:1041200080F89C32F7E708B590F89C32DBB2032B9D
:1041300001D0002008BDD0F8B832002BF9D0DB69DF
:10414000002BF6D09847F4E708B5D0F8D432AE3358
:1041500050F823205AB190F89C32DBB2032B01D0E7
:10416000002008BD136A23B198470020F9E7032017
:10417000F7E70020F5E708B5D0F8D432AE3350F8B1
:1041800023205AB190F89C32DBB2032B01D00020DF
:1041900008BD536A23B198470020F9E70320F7E7E9
:1041A0000020F5E70020704708B5012380F89C3215
:1041B000D0F8B83223B15B680179984710B908BDCF
:1041C0000020FCE70320FAE700207047002070473A
:1041D00038B504460D46002945D1D0F89432032B5A
:1041E00001D0084638BDD0F85831B0F8602193426C
:1041F00009D890F8AA3203F01F03012B12D0022B2A
:104200001FD0084613E09B1AC0F85831D0F864114B
:104210001144C0F864119A4238BF1A4600F08EFC6F
:104220002846DFE790F8AE12FFF7CEFF20B994F8EA
:104230009C32DBB2032B09D0204600F087FC2846D5
:10424000D0E790F8AE12FFF7C1FFEFE700F1AE0341
:1042500054F823301A69002AEED0C4F8D4021B693E
:1042600020469847E8E701F07F01FFF7AFFF90B9DC
:1042700094F89C32DBB2032BB4D100F1AE0354F8B6
:1042800023309A69002AADD0C4F8D4029B6929462C
:1042900020469847A6E70020A4E738B504460D4617
:1042A00000294CD1D0F89432022B07D094F8A00208
:1042B00018B1002384F8A032284638BD8269038CE7
:1042C0009A420ED89A421AD094F89C32DBB2032B51
:1042D00029D080212046FDF795FF204600F041FCC3
:1042E000E4E7D21A8261416A1944416200F00DFC90
:1042F00000231A4619462046FDF7A4FFD6E7426977
:104300009342E1D8D0F898329A42DDD20022114689
:1043100000F0FBFB0021C4F898120B460A46204629
:10432000FDF790FFC2E7D4F8B832DA68002AD0D09F
:104330000022C4F8D422DB6820469847C9E741F040
:104340008001FFF743FF90B994F89C32DBB2032B56
:10435000B3D100F1AE0354F823305A69002AACD02F
:10436000C4F8D4025B69294620469847A5E7002097
:10437000A3E70B88027813440B8003781844704736
:10438000428803789A4218D930B583B004460D4666
:10439000ADF806306388BDF806209A420AD20DF1C6
:1043A0000601FFF7E6FF4378052BF3D18378AB4294
:1043B000F0D100E0002003B030BD0020704703467C
:1043C000002002E00130C0B201331A78002AF9D18E
:1043D00070470B7803704B7843708B78CA7843EA48
:1043E000022343800B794A7943EA022383808B7945
:1043F000CA7943EA0223C380704710B5044680217E
:10440000FDF700FF00212046FDF7FCFE10BD30B592
:1044100083B004460D460023ADF806304A88130ADF
:10442000013B062B00F2AB80DFE803F0041F33A949
:10443000A98D9A00D0F8B4321B680DF10601007CFA
:104440009847EA88002A00F0A380BDF80630002BC8
:1044500000F099809A4228BF1A46ADF8062001461E
:10446000204600F044FB03B030BD037C43B9D0F8D4
:10447000B8329B6A0DF10600984702234370E0E7CB
:10448000D0F8B832DB6A0DF106009847022343707A
:10449000D7E7D2B2052A52D8DFE802F003101D2A6E
:1044A0003744D0F8B4325B6823B10DF10601007CCB
:1044B0009847C6E72946FFF7A0FFD4E7D0F8B43203
:1044C0009B6823B10DF10601007C9847B9E72946A6
:1044D000FFF793FFC7E7D0F8B432DB6823B10DF1E3
:1044E0000601007C9847ACE72946FFF786FFBAE74C
:1044F000D0F8B4321B6923B10DF10601007C984756
:104500009FE72946FFF779FFADE7D0F8B4325B6942
:1045100023B10DF10601007C984792E72946FFF789
:104520006CFFA0E7D0F8B4329B6923B10DF106010E
:10453000007C984785E72946FFF75FFF93E7294608
:10454000FFF75BFF8FE7037C33B9D0F8B8325B6BC2
:104550000DF10600984774E72946FFF74EFF82E702
:10456000037C43B9D0F8B8321B6B0DF106009847B5
:104570000723437065E72946FFF73FFF73E72946A6
:10458000FFF73BFF6FE729462046FFF736FF6AE754
:10459000204600F0DBFA66E738B504468B88FBB9A5
:1045A000CB88EBB94B887F2B1AD803F07F0590F8A6
:1045B0009C32DBB2032B0CD080F89E522946FDF7CB
:1045C00031FE204600F0C2FA35B1022384F89C3255
:1045D00009E0FFF712FF06E0012384F89C3202E0B5
:1045E0002046FFF70AFF38BD70B504460E468D78A9
:1045F0002F4B1D70012D10D890F89C32DBB2022B8E
:104600000FD0032B26D0FFF7F8FE294B1978204650
:10461000FFF702FD0325284670BDFFF7EEFE0325D8
:10462000F9E7A5B145602946FFF7EDFC054638B12D
:1046300031462046FFF7E1FE022384F89C32EAE788
:10464000204600F083FA032384F89C32E3E700F06D
:104650007DFAE0E7CDB141688D4225D0C9B2FFF7C0
:10466000DBFC134B197861602046FFF7CCFC054654
:10467000B0B131462046FFF7C0FE21792046FFF752
:10468000CBFC022384F89C32C5E7022380F89C32DD
:1046900045602946FFF7C0FC204600F057FABAE70C
:1046A000204600F053FAB6E700F050FA0025B2E7D2
:1046B000581E002008B5CB88012B0BD190F89C32F6
:1046C000DBB2022B09D9032B11D10122011D00F00D
:1046D0000EFA01E0FFF791FE08BD5BB23BB1014667
:1046E000002341F8083F012200F001FAF4E7FFF748
:1046F00084FEF1E708B590F89C32013B022B12D8FA
:10470000CB88022B0CD10123C360D0F8A4320BB1AB
:104710000323C360022200F10C0100F0E8F908BD98
:10472000FFF76BFEFBE7FFF768FEF8E708B54B887D
:10473000012B04D0022B07D0FFF75FFE08BDC0F8A5
:10474000A43200F003FAF9E78B881B0A80F8A03244
:1047500000F0FCF9F2E708B590F89C32013B022B1F
:1047600009D84B88012B00D008BD0023C0F8A43223
:1047700000F0ECF9F8E7FFF740FEF5E738B50C7804
:1047800004F06004202C06D0402C04D06CB1FFF75C
:1047900034FE002407E0D0F8D432AE3350F8233092
:1047A0009B6898470446204638BD4D78092D1DD892
:1047B000DFE805F012191C161C08051C0F0BFFF78B
:1047C00026FEF0E7FFF7E8FEEDE7FFF70DFF0446F2
:1047D000E9E7FFF76FFFE6E7FFF78CFF2C46E2E71C
:1047E000FFF7A4FFDFE7FFF7B6FFDCE7FFF705FE03
:1047F000D9E770B505460C460B7803F06003202B13
:1048000007D0402B05D023B1FFF7F7FD0026304637
:1048100070BD95F89C32013B022B26D821790129E5
:1048200005D921462846FFF7E8FD0026EFE7284690
:10483000FFF7CAFC68B900F1AE0255F82220916872
:1048400089B1C5F8D40293682146284698470646A0
:1048500000E00326E388002BD9D1002ED7D12846CB
:1048600000F074F9D3E70326F4E721462846FFF762
:10487000C4FD0026CBE72DE9F04106460D468B88A6
:10488000DFB20C7804F06004202C08D0402C06D055
:10489000DCB1FFF7B2FD00242046BDE8F0813946C7
:1048A0003046FFF793FC0446002840F0F980C6F834
:1048B000D40200F1AE0356F823309B68002BEBD0F6
:1048C0002946304698470446E6E791F80180B8F15A
:1048D000010F31D0B8F1030F05D0B8F1000F67D048
:1048E000FFF78BFDD8E790F89C32DBB2022B04D0A7
:1048F000032B12D0FFF781FDCEE70FB1802F04D13B
:1049000029463046FFF779FDC6E73946FDF77AFCC0
:1049100080213046FDF776FCBEE74B8823B91FB1F6
:10492000802F01D0CB881BB1304600F00FF9B3E7E0
:104930003946FDF767FCF7E790F89C32DBB2022BB3
:1049400004D0032B12D0FFF758FDA5E70FB1802F3D
:1049500004D129463046FFF750FD9DE73946FDF763
:1049600051FC80213046FDF74DFC95E74B88002B2C
:1049700092D117F07F0F17D1304600F0E7F8394693
:104980003046FFF723FC002886D1C6F8D40200F198
:10499000AE0256F822209268002A00F08380294651
:1049A00030469047044677E73946FDF733FCE3E7A6
:1049B00090F89C22D2B2022A05D0032A28D0FFF711
:1049C0001CFD444668E70FB1802F14D113F0800F0F
:1049D00015D107F07F0707EB8707B90001F5A8712C
:1049E00031440431002301F80E3F0222304600F02A
:1049F0007EF8444650E7FFF700FD44464CE707F0D9
:104A00007F0707EB8707B900103131440431E9E72C
:104A10005BB2002B20DB07F00F0202EB820200EBFF
:104A2000820292F8634124B3002B25DB07F07F0359
:104A300003EB83039C0004F5A874344404340FB1E1
:104A4000802F22D10023A373022204F10E013046ED
:104A500000F04DF844461FE707F00F0202EB820218
:104A600000EB820292F82340002CDDD1FFF7C5FC59
:104A700012E7FFF7C2FC0FE707F07F0303EB8303A6
:104A80009C00103434440434D9E739463046FDF7ED
:104A900073FB10B10123A373D6E70023A373D3E7FD
:104AA0000024F9E60446F7E600B370B50D46164655
:104AB0000446FFF784FC01304300B3F5007F06D8BD
:104AC0009BB233802B7003236B7002230AE04FF4F8
:104AD0000073F6E7EA5401345A1CD2B20021A954FB
:104AE0000233DBB22278002AF4D170BD704708B5DA
:104AF00013460222C0F894224361416283610A4650
:104B00000021FDF797FB002008BD08B513460A46B3
:104B10000021FDF78FFB002008BD08B513460322D6
:104B2000C0F89422C0F85431C0F86411C0F858316C
:104B30000A460021FDF786FB002008BD08B5134694
:104B40000A460021FDF77EFB002008BD08B50422BF
:104B5000C0F8942200231A461946FDF76BFB00208B
:104B600008BD08B50522C0F8942200231A4619464C
:104B7000FDF768FB002008BD10B5D0F8D43203F172
:104B8000B00250F822408CB100EB820043687BB148
:104B900094F80002FF280DD09B6894F8012221466A
:104BA0009847FF2384F80032002010BD0320FCE763
:104BB0000020FAE70020F8E70A2303800048704746
:104BC00010010020F8B506460F4F82213846FFF746
:104BD000D7FB054601213846FFF7D2FB0446812169
:104BE0003846FFF7CDFB0DB11022AA711CB140224F
:104BF00022710022627118B14022027100224271BA
:104C0000432333800048F8BD94000020F8B50646E1
:104C10000F4F82213846FFF7B3FB05460121384686
:104C2000FFF7AEFB044681213846FFF7A9FB0DB123
:104C30001022AA711CB1402222710022627118B1A7
:104C40004022027100224271432333800048F8BDA4
:104C500094000020F8B506460F4F82213846FFF732
:104C60008FFB054601213846FFF78AFB0446812168
:104C70003846FFF785FB0DB11022AA711CB1002246
:104C800022710222627118B1002202710222427165
:104C9000432333800048F8BD9400002038B5D0F895
:104CA000D432B03350F8235095B10446FDF77AFA68
:104CB000C5F80C02D4F8D432B03304EB8304636833
:104CC000DB6805F50371D5F804029847002038BD6C
:104CD0000320FCE738B5D0F8C852D0F8D432B0334E
:104CE00050F8234084B301F00F0303EB830200EB81
:104CF000820252694AB103EBC30C05EB8C05ED69E6
:104D0000B2FBF5FC05FB1C2292B10023C4F814325F
:104D1000D0F8D432B03300EB830043681B69ABB1E9
:104D20000A4604F50471D4F808029847002038BDFB
:104D300003EB830300EB830300245C6123462246DC
:104D4000FDF778FA2046F2E70320F0E70020EEE7CF
:104D5000F0B583B0D0F8D43203F1B00250F822702D
:104D600000228DF80720ADF80420002F7BD00446E8
:104D70000D46097811F0600634D0202E6CD1EA88F7
:104D80002AB311F0800F07D16B7887F80032EA88D8
:104D90003F2A13D8D2B212E0B03300EB83035B6832
:104DA0009B68394668789847EA88072A28BF07220F
:104DB00039462046FFF79BFE002651E0402287F847
:104DC000012239462046FFF7A8FE002648E0B0330E
:104DD00000EB83035B689B6800222946687898474C
:104DE00000263DE06F780B2F31D8DFE807F0063959
:104DF0003030303030303030162690F89C32DBB214
:104E0000032B04D02946FFF7F8FA032628E00222F4
:104E100001A9FFF76CFE3E4622E090F89C32DBB21F
:104E2000032B04D02946FFF7E8FA032618E00122F5
:104E30000DF10701FFF75BFE12E090F89C32DBB248
:104E4000032B0DD02946FFF7D8FA032608E02946A0
:104E5000FFF7D3FA032603E02946FFF7CEFA03262D
:104E6000304603B0F0BD0326FAE738B50446812189
:104E7000FDF7C0F9002584F8375001212046FDF7E1
:104E8000B9F984F8775182212046FDF7B3F984F807
:104E90004B506564D4F8D43203F1B00254F82220A8
:104EA0009AB1B03304EB83035B685B689847D4F82E
:104EB000D432B03354F82300FDF77EF9D4F8D4325D
:104EC000B03344F82350C4F8BC52002038BD70B54C
:104ED00004464FF40770FDF76BF9002849D00546EA
:104EE0004FF407720021FBF7CFF9D4F8D432B03376
:104EF00044F82350C4F8BC52237C002B41D14FF41A
:104F00000073022281212046FDF769F9012684F809
:104F100037604FF40073022231462046FDF75FF9F7
:104F200084F87761102363640823032282212046DA
:104F3000FDF755F9012384F84B300026C5F80462CB
:104F4000D4F8D432B03304EB83035B681B68984712
:104F5000C5F81462C5F81862D5F8042262B3257C3E
:104F60001DBB4FF4007301212046FDF76BF9284665
:104F700070BDD4F8D432B033002244F82320022587
:104F8000F5E74023022281212046FDF728F901267A
:104F900084F837604023022231462046FDF71FF98E
:104FA00084F8776110236364BEE740230121204623
:104FB000FDF748F90025DAE70225D8E739B1D0F83E
:104FC000D432B03300EB83004160002070470320EF
:104FD0007047D0F8D432B03350F823302BB1C3F837
:104FE0000812C3F810220020704703207047D0F841
:104FF000D432B03350F823301BB1C3F80412002070
:1050000070470320704708B5D0F8D432B03350F859
:1050100023208AB1D2F814320BB1012008BD01233C
:10502000C2F81432D2F810328362D2F808228121F9
:10503000FDF700F90020F1E70320EFE710B5D0F805
:10504000D432B03350F8232092B1047C44B94FF4E9
:105050000073D2F804220121FDF7F4F8204610BDB8
:105060004023D2F804220121FDF7ECF80024F5E7F3
:105070000324F3E7DFF834D0FCF78CFE0C480D492D
:105080000D4A002302E0D458C4500433C4188C42A3
:10509000F9D30A4A0A4C002301E013600432A24209
:1050A000FBD3FBF7C9F8FBF743FC70470000032074
:1050B000000000201C010020505100081C010020AD
:1050C0005C1E0020FEE70000F8B500BFF8BC08BC7D
:1050D0009E467047F8B500BFF8BC08BC9E467047B6
:1050E0000006101600061016000000000000000068
:1050F000010203040607080953544D333220566950
:10510000727475616C20436F6D506F727400000093
:1051100053544D6963726F656C656374726F6E6929
:105120006373000043444320436F6E666967000069
:1051300043444320496E74657266616365000000F4
:08514000BCB2FF7F010000007A
:045148001902000840
:04514C00F101000865
:10515000737470203F3F3F3F3F3F20203F3F3F3F22
:105160003F3F3F3F3F3F0D0A53776565705F737464
:105170006172740A0D000100100000000024F400A8
:105180001A03000000000000000000000000000002
:1051900000000000000000000000000004030904FB
:1051A0001201000202020040830440570002010283
:1051B00003010000FD1D0008091E0008CD1E0008A7
:1051C000A91E0008951E0008E91E00080D1F000812
:1051D000591F0008311F0008351F00083D1F000837
:1051E000391F000809024300020100C0320904000F
:1051F0000001020201000524001001052401000144
:105200000424020205240600010705820308001099
:1052100009040100020A0000000705010240000025
:105220000705810240000000CF4E00086B4E0008C9
:10523000514D000800000000794B0008D54C0008D3
:105240009D4C00080000000000000000000000006D
:10525000554C00080D4C0008C54B0008B94B000820
:0C5260000A0600020000004001000000EF
:04000005080050752A
:00000001FF
